:100000000C944A000C94DA1E0C94DA1E0C949E1682
:100010000C94DA1E0C94DA1E0C94AA1A0C94DA1EB4
:100020000C94DA1E0C94DA1E0C94781C0C94DA1ED4
:100030000C94DA1E0C94461D0C94DA1E0C94DA1EF5
:100040000C94DA1E0C94B41B0C94DA1E0C94DA1E79
:100050000C94DA1E0C94DA1E0C94DA1E0C94DA1E40
:100060000C941C1B0C94DA1E0C940B1C0C94DA1EC2
:100070000C94DA1E0C94DA1E9A00C700E6003302D4
:100080006402C302F402410338003860003DC23804
:10009000603A678011241FBECFEFCDBFDFE3DEBF24
:1000A000E8E8F0E040E017C0B591A59135912591C1
:1000B000059107FD0CC095918591EF01F92FE82F6F
:1000C00005900D92A217B307D9F7FE0104C01D9247
:1000D000A217B307E1F7E439F40731F70E94541986
:0800E0000C943E1EF894FFCFC2
:1000E8002F923F924F925F926F927F928F929F9240
:1000F800AF92BF92CF92DF92EF92FF920F931F932E
:10010800CF93DF93CDB7DEB7A197CDBFDEBF8DB656
:100118009EB6E091603A8E2F90E08830910508F005
:1001280013C5FC01E45CFF4F0C94B61E8091613A44
:10013800843008F46AC564E0CE0101960E94E41A8E
:10014800FE0131969E012B5F3F4F90E081918B31EC
:1001580009F49F5F2E173F07C9F7943019F01092E2
:10016800613A53C582E39CE880935C3A90935D3A88
:1001780010E0812F0E94701A1F5F1C30D1F781E0B8
:100188008093603A42C58091613A882309F43DC55D
:100198000E94991C182F898340915C3A50915D3ACE
:1001A80061E0CE0101960E94F31C80935C3A909323
:1001B8005D3A1B3119F0173709F027C582E08093A3
:1001C800603A23C58091613A873008F41EC567E01C
:1001D800CE010D960E94E41A40915C3A50915D3A26
:1001E80065E0CE010D960E94F31CBC0180935C3A39
:1001F80090935D3AFE013D969E01205F3F4F50E08F
:1002080091919B3109F45F5FE217F307C9F7533007
:1002180009F0EAC08B8990E0982F88272A89822BD9
:100228006817790709F0D6C088E20E94210680E5A0
:100238000E94210688E70E94210619821A821B82E1
:100248001C821D821E821F8218869E012F5F3F4FCF
:1002580044E065E370E281E00E94F80A9E01245EB2
:100268003F4F41E069E370E281E00E94A613E0E4B9
:10027800F1E040855185242F352F40E050E060E0C3
:1002880070E080E090E0A980BA80CB80DC80ED80CF
:10029800FE800F8118850E94641E29833A834B8350
:1002A8005C836D837E838F8398874085518528EE94
:1002B80033E0429FC001439F900D529F900D11243F
:1002C8008A8F9B8F8C8D9D8D892B49F09E01265E90
:1002D8003F4F41E064E370E281E00E9453149E01C5
:1002E8002F5F3F4F44E065E370E281E00E94EE0F2C
:1002F80010924801109249019E01285E3F4F41E04B
:100308006AE370E281E00E94A613888D998D892B9B
:1003180009F04CC09E012C5E3F4F42E06CE170E05A
:1003280080E00E94220F2C893D894E895F8937FF22
:100338001FC0A6EFBFEF0E94811E6C8B7D8B8E8B3A
:100348009F8B9E012C5E3F4F42E062E070E080E0B0
:100358000E94F3121C8A1D8A1E8A1F8A9E012C5E27
:100368003F4F42E060E070E080E00E94F3121EC060
:10037800AAE0B0E00E94331E6C8B7D8B8E8B9F8B26
:100388009E012C5E3F4F42E060E070E080E00E94FA
:10039800F3121C8A1D8A1E8A1F8A9E012C5E3F4FFB
:1003A80042E062E070E080E00E94F31281E090E0B9
:1003B8008C8B9D8B9E012C5E3F4F41E067E470E281
:1003C8000E94531410E0812F0E94A1191F5F1B3057
:1003D800D1F707C010E0812F0E94701A1F5F1C30F0
:1003E800D1F71092603A11C4AB0162E0CE01429697
:1003F8000E94F31C80935C3A90935D3A088910E060
:1004080020E030E09801112700278A89082B898984
:1004180090E0982F8827092E000CAA0BBB0B082BFD
:10042800192B2A2B3B2B81E08093603A90915F3AFD
:10043800EEEFFDEA80E0A3E04081518162817381A3
:10044800041715072607370719F4A093603A982F61
:100458008F5F3996853181F790935F3AD6C3809143
:10046800613A882309F4D1C30E94AA1E182F1F706D
:100478008DB79EB7811B91098DBF9EBFADB7BEB723
:1004880011967D01812F0E94FE1D811116C0612FDA
:10049800C7010E94E41A40915C3A50915D3A612F7D
:1004A800C7010E94F31C80935C3A90935D3A84E004
:1004B8008093603A8DBE9EBEA8C38DBE9EBEA5C366
:1004C8008091613A882309F4A0C30E94991C182FCF
:1004D8008C8B40915C3A50915D3A61E0CE01449634
:1004E8000E94F31C7C0180935C3A90935D3A12372A
:1004F80009F041C082E00E94FE1D811186C362E0BE
:10050800CE010D960E94E41AA70162E0CE010D9675
:100518000E94F31C8C0180935C3A90935D3A8E851F
:100528008330A9F48CE00E94FE1D81116EC36CE03B
:10053800CE0101960E94E41AA8016CE0CE01019652
:100548000E94F31C80935C3A90935D3A14C085E056
:100558000E94FE1D811159C365E0CE0101960E94DB
:10056800E41AA80165E0CE0101960E94F31C80936D
:100578005C3A90935D3A85E08093603A46C38091F7
:10058800613A882309F441C30E94AA1E182F1F70DC
:10059800EDB7FEB7E11BF109EDBFFEBF8DB79EB702
:1005A80001967C01812F0E94FE1D811116C0612FCA
:1005B800C7010E94E41A40915C3A50915D3A612F5C
:1005C800C7010E94F31C80935C3A90935D3A86E0E1
:1005D8008093603A8DBE9EBE18C38DBE9EBE15C365
:1005E8008091613A882309F410C3CDB6DEB60E9423
:1005F800AA1E182F1F70ADB7BEB7A11BB109ADBF9A
:10060800BEBFEDB7FEB731967F01812F0E94FE1D58
:10061800811130C0612FC7010E94E41A40915C3AF1
:1006280050915D3A612FC7010E94F31C80935C3A98
:1006380090935D3A1230A8F080915F3A90E0FC0107
:10064800EE0FFF1FEE0FFF1FEE0FFF1F8E0F9F1FF6
:10065800FC01E250F2459085D70111968C91890FE3
:1006680001C080E080935E3A87E08093603ACDBE17
:10067800DEBECBC28DBE9EBEC8C28091613A8230BA
:1006880008F4C3C262E0CE010D960E94D71C8D8586
:1006980088230CF082C29E8599230CF074C250C244
:1006A800EDB7FEB7EB19F109EDBFFEBF8DB79EB7E9
:1006B80001966C012C0190E29B15D0F4BB2009F146
:1006C8008601EE24EA94EB0CF12CAFEFEA1AFA0A51
:1006D800EC0CFD1C81E00E94FE1D811112C00E94DD
:1006E800991CF80181938F01EE16FF0699F709C04E
:1006F8008B2D0E94FE1D811120C26B2DC6010E9408
:10070800E41A40915C3A50915D3A6B2DC6010E9403
:10071800F31C80935C3A90935D3AD6019C91892FA3
:10072800807F803519F0803609F0B6C194FF0AC081
:10073800F6018181082E000C990B892F881F8827C4
:10074800881F01C080E0EB2CF12CF1E0EF1AF108D2
:1007580088A319821A821B821C821D821E821F8214
:100768001886EFEFEB0D09F41DC2712CA12CB12CEA
:10077800C12CD12C612C1E8EF0E08E2F90E09201BE
:10078800280F391FD9012C918701081B190B000F5D
:10079800111F000F111F000F111F30E040E050E043
:1007A80060E070E080E090E00E94791D722AA32A40
:1007B800B42AC52AD62A672ABE8DB82BBE8FF92B34
:1007C800E150D9F67982AA82BB82CC82DD826E8220
:1007D800BF83F887E8A1EE2309F4B9C18701000FA8
:1007E800111F000F111F000F111F2FEF3FEF4FEFC9
:1007F8005FEF6FEF7FEF8FEF9FEF0E94791DE98129
:10080800E22BFA81F32BBB81B42B1C81152B0D81B4
:10081800062BFE80F72AEF80E82AD884D92AE983B4
:10082800FA83BB831C830D83FE82EF82D8862E2F2A
:100838003F2F4B2F512F602F7F2D8E2D9D2DA0E008
:100848000E94271E09F4CEC1B1C12E2F3F2F4B2F76
:10085800512F602F7F2D8E2D9D2D0E94DF1D298306
:100868003A834B835C836D837E838F8398871614CA
:100878006CF1ABC129813A814B815C816D817E81AC
:100888000F2EFAE0AF2EF02DB12CC12CD12CE12C7B
:10089800F12C00E010E08F8198850E940E1E522EE8
:1008A8003E8FB42FF52FE62F472E8F8F99A32983DC
:1008B8003A834B835C836D837E838F839887A0E024
:1008C8000E94271E09F46FC0712C5FC029813A81EC
:1008D8004B815C816D817E818F819885E0E001E0AC
:1008E8000E94791D2E8F432E542E752E6F8FB72F91
:1008F800A82FF92F02E00E94791DA22EB32EC42E34
:10090800D52EE62EF72E082F192F2E8D342D452D96
:10091800572D6F8D7B2F8A2F9F2F0E94641EEF5FAC
:10092800E615ECF229833A834B835C836D837E83DF
:100938008F83988738C00F2EFAE0AF2EF02DB12C98
:10094800C12CD12CE12CF12C00E010E0252D3E8D9E
:100958004B2F5F2F6E2F742D8F8D99A10E940E1E25
:10096800522E3E8FB42FF52FE62F472E8F8F99A347
:10097800A0E00E94271E49F419821A821B821C8259
:100988001D821E821F8218860EC07A947610D3CFDD
:1009980059822E8D2A83BB83FC83ED834E82BF8DC3
:1009A800BF83E9A1E887F8A1FF2309F45DC080911E
:1009B8005F3A90E0FC01EE0FFF1FEE0FFF1FEE0FF6
:1009C800FF1F8E0F9F1FFC01E250F245878184FFB5
:1009D80016C029813A814B815C816D817E818F812E
:1009E80098850E94DF1D29833A834B835C836D833E
:1009F8007E838F83988703C028A12223A9F1E091E1
:100A08005F3A89E0E89FF0011124E250F2458781BE
:100A180085FF2AC0D980EA80FB800C811D81BE81B8
:100A2800FF81E8852D2D3E2D4F2D502F612F7B2FD7
:100A38008F2F9E2FA0E00E94271E21F080915E3A02
:100A4800811112C02D2D3E2D4F2D502F612F7B2F40
:100A58008F2F9E2F0E94DF1D29833A834B835C834F
:100A68006D837E838F83988780915F3A90E0FC0145
:100A7800EE0FFF1FEE0FFF1FEE0FFF1FE80FF91F0E
:100A8800E250F245648175819E012F5F3F4F468198
:100A980080E00E94EE0F4EC080915F3A90E0FC012A
:100AA800EE0FFF1FEE0FFF1FEE0FFF1F8E0F9F1F92
:100AB800FC01E250F24580819181A281B3818115C8
:100AC800E1E09E07E0E6AE07B10521F00997A10530
:100AD800B10581F500E010E0D60111968C911197CF
:100AE80090E0982F882712962C91822B89839A83DD
:100AF80080915F3A90E0FC01EE0FFF1FEE0FFF1FA1
:100B0800EE0FFF1F8E0F9F1FFC01E250F24564811C
:100B18007581600F711F9E012F5F3F4F41E081E09B
:100B28000E9453140F5F1F4FB2E0CB0ED11C05304B
:100B3800110591F62DBE3EBE03C02DBE3EBE65C05A
:100B480081E08093603A61C01092603A5EC029816A
:100B58003A814B815C816D817E818F819885A0E08F
:100B68000E94271E41F580CF16140CF4AFCE29C081
:100B78002DB63EB6EE85EF70F0E18F9FC0011124CF
:100B8800BE2EB82A8DCD982F9077903789F7D8CF79
:100B98002DB63EB68F70B82E83CD982F90779037AC
:100BA80079F2F6CF28A1211119CE5ECF60905E3A76
:100BB80061104BCE21CF60905E3A662009F41CCFBD
:100BC800D3CF66200CF456CE4FCF66200CF452CE0D
:100BD800EECED980EA80FB800C811D81BE81FF8129
:100BE800E88530CF80915F3A90E0FC01EE0FFF1F5F
:100BF800EE0FFF1FEE0FFF1F8E0F9F1FFC01E2502D
:100C0800F245878185FF30CFE4CF8DBE9EBEA19689
:100C1800CDBFDEBFDF91CF911F910F91FF90EF9075
:100C2800DF90CF90BF90AF909F908F907F906F9004
:0A0C38005F904F903F902F900895B9
:100C42002F923F924F925F926F927F928F929F92DA
:100C5200AF92BF92CF92DF92EF92FF920F931F93C8
:100C6200CF93DF93CDB7DEB7E497CDBFDEBF182FAA
:100C7200882E912CB4016C5E7F4F9E012F5F3F4FF7
:100C820042E080E00E94220FB4016A5E7F4F9E0123
:100C92002B5F3F4F42E080E00E94220F89819A81C0
:100CA200AB81BC81892B8A2B8B2B09F4F3C28D81FA
:100CB2009E81AF81B885892B8A2B8B2B09F4EAC2DE
:100CC200183719F06AE170E002C06CE170E0680D5B
:100CD200791D9E012F5D3F4F41E080E00E94A613E7
:100CE20009A11AA1B80181E00E94B9176C01990FFC
:100CF200EE08FF08CD8EDE8EEF8EF8A2B80180E0FE
:100D02000E94B9172C01990F66087708CC24F7FCCA
:100D1200C394DD24EE24FF24AC2CAA0CABAA2A2C0B
:100D2200312C8101005F1F4F0BA71CA79E01275E7C
:100D32003F4F42E0B80180E00E94220F89819A81F0
:100D4200AB81BC815C016D01E12CF12C87018BA38D
:100D5200BCA2CDA2DEA2EFA2F8A609A71AA70D8116
:100D62001E812F813885A02EB12EC22ED32EE12CCA
:100D7200F12C00E010E02BA13CA14DA15EA160E0AE
:100D820070E080E090E00E940419205B3C434F4FEA
:100D92005F4F6F4F7F4F8F4F9F4F0F2EF0EAAF2E57
:100DA200F02D0F2EF6E8BF2EF02DCC24C394D12CBB
:100DB2000E940E1E822F932FA42FB52F8D8B9E8BF8
:100DC200AF8BB88F498D5A8D6B8D7C8D840F951F9B
:100DD200A61FB71F898F9A8FAB8FBC8FB401605F3C
:100DE2007F4F620D731D9E012B5E3F4F42E080E0FC
:100DF2000E94F3129E01275E3F4F42E06BA57CA545
:100E020080E00E94F3128D8D9E8DAF8DB8A1892B4B
:100E12008A2B8B2B09F49EC1DBA8CD2CD12CCBAA1B
:100E2200DCAA9E012F5E3F4F42E0B60180E00E94A5
:100E3200220FED8CFE8C0F8D18A1EBA2FCA20DA34C
:100E42001EA31E141F04100611060CF05CC089813B
:100E52009A81AB81BC818C019D0140E050E0BA01D6
:100E62008BA71CA72DA73EA74FA758AB69AB7AABA0
:100E72000D811E812F813885A02EB12EC22ED32E38
:100E8200E12CF12C00E010E02BA53CA54DA55EA5C0
:100E920060E070E080E090E00E940419ABA0BCA08A
:100EA200CDA0DEA0DD0CAA08BA2C6501ABA6BCA6BB
:100EB200CDA6DEA6ABA0BCA0CDA0DEA0EBA4FE2CEE
:100EC2000E2D1E2D0E9404193B594243524E6F4F64
:100ED2007F4F8F4F9F4FA12C0F2EFAECBF2EF02D7C
:100EE2000F2EFAE9CF2EF02D0F2EFBE3DF2EF02D81
:100EF200E12CF12C00E010E00E940E1E2D873E87AF
:100F02004F87588B65C089819A81AB81BC816C0106
:100F12007D0100E010E098018BA7DCA6EDA6FEA6FD
:100F22000FA718AB29AB3AAB0D811E812F813885F3
:100F3200A02EB12EC22ED32EE12CF12C00E010E017
:100F42002BA53CA54DA55EA560E070E080E090E099
:100F52000E940419EBA0FCA00DA11EA11095009502
:100F6200F094E094E11CF11C011D111D5701680170
:100F7200DD0CAA08BA2C6501ABA2BCA2CDA2DEA2EE
:100F8200AE2CBF2CC02ED12EEBA0FE2C0E2D1E2D72
:100F92000E9404193B594243524E6F4F7F4F8F4F6D
:100FA2009F4FA12C0F2EFAECBF2EF02D0F2EFAE937
:100FB200CF2EF02D0F2EFBE3DF2EF02DE12CF12CA6
:100FC20000E010E00E940E1E2D873E874F87588B4F
:100FD20049895A896B897C898D859E85AF85B889B7
:100FE200840F951FA61FB71F898B9A8BAB8BBC8B67
:100FF200B401620D731D9E01235F3F4F42E080E00A
:101002000E94F3129E012F5E3F4F42E06BA97CA922
:1010120080E00E94F3128D8D9E8DAF8DB8A11816BF
:1010220019061A061B068CF4BC01CD016B5F7F4FBB
:101032008F4F9F4F2AE030E040E050E00E94921D27
:101042002D8F3E8F4F8F58A310C0BC01CD0165502C
:101052007109810991092AE030E040E050E00E94E4
:10106200921D2D8F3E8F4F8F58A389899A89AB8904
:10107200BC896C017D018BA3DCA2EDA2FEA2282F0C
:101082003D2D4E2D5F2D60E070E080E090E002E0AB
:101092000E94791DA22EB32EC42ED52EE62EF72E37
:1010A200E82F192F05E00E94791D0E2F0E946D1E58
:1010B200ABA0BCA0CDA0DEA0E12CF12C00E010E0A2
:1010C2000E94641E03E00E94791DE98CFA8C0B8D4C
:1010D2001C8D6701780156016701E12CF12C870113
:1010E200ABA2BCA2CDA2DEA2EFA2F8A609A71AA7C4
:1010F200E12CF12C00E010E00E940E1E822F932FB3
:10110200A42FB52F89879A87AB87BC874D8D5E8DBB
:101112006F8D78A177235CF4B095A0959095819519
:101122009F4FAF4FBF4F89879A87AB87BC879E017E
:10113200235E3F4F42E0B401685E7F4F80E00E9431
:10114200F3129E01275F3F4F42E068E170E080E0CA
:101152000E94F312411451046104710409F49AC00B
:1011620054F47094609450944094411C511C611C3E
:10117200711C62E001C060E0262E312C81010C5FFF
:101182001F4F0BA71CA79E01235F3F4F42E0B801F0
:1011920080E00E94220F89819A81AB81BC815C012F
:1011A2006D01E12CF12C87018BA3BCA2CDA2DEA2A2
:1011B200EFA2F8A609A71AA70D811E812F813885F3
:1011C200A02EB12EC22ED32EE12CF12C00E010E085
:1011D2002BA13CA14DA15EA160E070E080E090E017
:1011E2000E94041973016201FF0CCC08DC2C760109
:1011F200CBA2DCA2EDA2FEA2A42CB52CC62CD72C2D
:10120200EBA0FE2C0E2D1E2D0E9404193B594243C9
:10121200524E6F4F7F4F8F4F9F4FA12C0F2EFAECE4
:10122200BF2EF02D0F2EFAE9CF2EF02D0F2EFBE35D
:10123200DF2EF02DE12CF12C00E010E00E940E1EBA
:10124200822F932FA42FB52F89879A87AB87BC87CC
:101252004D855E856F857889840F951FA61FB71F00
:101262008D879E87AF87B88B9E01235F3F4F42E0F9
:101272006BA57CA580E00E94F31204E0800E911C15
:10128200B401620D731D9E01275F3F4F42E080E073
:101292000E94F312E496CDBFDEBFDF91CF911F9182
:1012A2000F91FF90EF90DF90CF90BF90AF909F9003
:1012B2008F907F906F905F904F903F902F90089506
:1012C2004F925F926F927F928F929F92AF92BF9254
:1012D200CF92DF92FF920F931F93CF93DF93CDB7FD
:1012E200DEB72897CDBFDEBF8C01B62ECDB6DEB6F7
:1012F200FC01F0808091633AF81242C14FEF5FEF38
:10130200C8010E940F1D892B09F03CC1F8016181BF
:10131200633019F0603109F008C1F801228130E030
:10132200322F22278381282B8480912C982C882489
:101332008581882A5901A80CB91CF1E0AF1AB108BD
:10134200E0E0F8E380E090E02C0140815181241735
:10135200350708F4E3C0A281B381AA15BB0508F4DE
:10136200DDC0633009F065C06DB67EB6880C991C8D
:10137200C40105966DB77EB7681B790B6DBF7EBF42
:101382000DB71EB70F5F1F4FC801EDB7FEB7F18251
:1013920033E0F80131838282241BE22FF0E0A41AA9
:1013A200B50AAE16BF0628F1B201660F771F660FA7
:1013B200771F660F771FDB01A050B84C14964D9132
:1013C2005C911597EE0FFF1FE40FF51FDC01A30FD1
:1013D200B11D61816C9361E0630FDC01A60FB11D49
:1013E2003E5F60816C932F5FE22FF0E0AE16BF0686
:1013F20048F763E0680D4FEF5FEFC8010E940F1DD1
:10140200F801E80DF91D8383948365E0680DC80136
:101412000E940E1819821A829E012F5F3F4F41E0EF
:1014220067E470E281E00E9453146DBE7EBE83E0E9
:10143200C9C08A3049F08B3009F0A6C0FCE3AF1670
:10144200F0E2BF0608F0A0C0241B822F90E0B50195
:10145200641B750B68177907E8F137E0B201660F74
:10146200771F660F771F660F771FFB01E050F84C5E
:101472004F01AF014C5F5F4F880F991FFA01A081A6
:10148200B181A80FB91FB801630F711DFB01608103
:101492001C9211966C93FA01A081B181A80FB91F19
:1014A20081E0830FB801680F711D3E5FFB0160810F
:1014B2008D919C911197862B8D939C932F5F822FF8
:1014C20090E0F40160817181F501E61BF70BE817EA
:1014D200F90790F6AE014F5F5F4F5A0188E0FA01BB
:1014E20011928A95E9F7F8018081898380E18A83E4
:1014F20082818B8383818C8384818D8385818E839A
:101502004FEF5FEF66E0C5010E940F1D8F83988742
:1015120068E0C5010E940E1880E154C00196389619
:101522008C30910509F010CF2FC0683069F4F801B2
:101532008281811109C08381811106C06B2DC8018E
:101542000E940E1888E03EC08E010F5F1F4F85E09B
:10155200F80111928A95E9F7F982862F80688A83C9
:1015620081E08B834FEF5FEF63E0C8010E940F1DA4
:101572008C839D8365E0C8010E940E1881E022C021
:1015820080E020C080E01EC0AE014F5F5F4F5A0175
:1015920085E0FA0111928A95E9F7F982862F80682F
:1015A2008A8382E08B834FEF5FEF63E0C5010E9485
:1015B2000F1D8C839D8365E0C5010E940E18F80102
:1015C20081818068CDBEDEBE2896CDBFDEBFDF91B1
:1015D200CF911F910F91FF90DF90CF90BF90AF906E
:0E15E2009F908F907F906F905F904F90089534
:1015F0002F923F924F925F926F927F928F929F9223
:10160000AF92BF92CF92DF92EF92FF920F931F9310
:10161000CF93DF9300D000D0CDB7DEB7F82E5B01BB
:10162000142F2B833C83D9011C9211961C92119785
:1016300012961C92129713961C92139714961C9252
:10164000149715961C92159716961C921697179636
:101650001C92642FC5010E942B1D8F3F09F4F3C01B
:10166000FF2009F464C0112309F4EDC0C12ED12C70
:10167000B1E0CB1AD108CC0CDD1CCC0CDD1CCC0CA1
:10168000DD1CCC0CDD1CA0E0B0E0E82EF12CC70185
:10169000880F991F880F991F880F991FFC01E05030
:1016A000F84C7F013496E983FA83F70180819181B8
:1016B000F501E81BF90BEA0FFB1F9F01220F331FF7
:1016C000E981FA8180819181F901E80FF91F808118
:1016D00091811C01282F332D40E050E060E070E044
:1016E00080E090E00C2D0E94791DEB81FC819080C0
:1016F000292920832181322B31832281422B42836D
:101700002381522B53832481622B64832581722B86
:1017100075832681822B86838781982B97831196E8
:10172000F0E1CF1AD108A11708F4BFCF8CC0E82E82
:10173000F12CF701EE0FFF1FEE0FFF1FEE0FFF1F43
:10174000E050F84C86819781892B09F47CC01123E5
:1017500009F479C0A12FB0E01197FD01E295F2954F
:10176000F07FFE27E07FFE27E983FA83E0E0F0E0E8
:10177000C701880F991F880F991F880F991F9C0117
:101780002050384C7901690136E0C30ED11CD701D5
:101790008D919C919501281B390BC9018E0F9F1FBC
:1017A000880F991FD6012D913C91820F931FDC0168
:1017B0002D903C90222D332D40E050E060E070E011
:1017C00080E090E009810E94791DAB81BC819C90F2
:1017D00029292C9311962C911197322B11963C9319
:1017E000119712962C911297422B12964C931297A6
:1017F00013962C911397522B13965C931397149670
:101800002C911497622B14966C93149715962C9127
:101810001597722B15967C93159716962C91169703
:10182000822B16968C93169717968C911797982B58
:1018300017969C933196A981BA815097A983BA8350
:10184000E11708F4A4CF2496CDBFDEBFDF91CF917E
:101850001F910F91FF90EF90DF90CF90BF90AF90CE
:101860009F908F907F906F905F904F903F902F90C0
:021870000895D9
:101872000000891112239B322446AD573665BF748E
:10188200488CC19D5AAFD3BE6CCAE5DB7EE9F7F83E
:101892008110080193331A22A5562C47B7753E646E
:1018A200C99C408DDBBF52AEEDDA64CBFFF976E81E
:1018B20002218B30100299132667AF763444BD554E
:1018C2004AADC3BC588ED19F6EEBE7FA7CC8F5D9FE
:1018D20083310A2091121803A7772E66B5543C452E
:1018E200CBBD42ACD99E508FEFFB66EAFDD874C9DE
:1018F20004428D5316619F702004A9153227BB360E
:101902004CCEC5DF5EEDD7FC6888E1997AABF3BABD
:1019120085520C4397711E60A1142805B3373A26ED
:10192200CDDE44CFDFFD56ECE9986089FBBB72AA9D
:1019320006638F7214409D512225AB343006B917CD
:101942004EEFC7FE5CCCD5DD6AA9E3B8788AF19B7D
:1019520087730E6295501C41A3352A24B1163807AD
:10196200CFFF46EEDDDC54CDEBB962A8F99A708B5D
:10197200088481951AA793B62CC2A5D33EE1B7F08D
:101982004008C919522BDB3A644EED5F766DFF7C3D
:10199200899400859BB712A6ADD224C3BFF136E06D
:1019A200C1184809D33B5A2AE55E6C4FF77D7E6C1D
:1019B2000AA583B4188691972EE3A7F23CC0B5D14D
:1019C2004229CB38500AD91B666FEF7E744CFD5DFD
:1019D2008BB502A499961087AFF326E2BDD034C12D
:1019E200C3394A28D11A580BE77F6E6EF55C7C4DDD
:1019F2000CC685D71EE597F42880A1913AA3B3B20D
:101A0200444ACD5B5669DF78600CE91D722FFB3EBC
:101A12008DD604C79FF516E4A9902081BBB332A2EC
:101A2200C55A4C4BD7795E68E11C680DF33F7A2E9C
:101A32000EE787F61CC495D52AA1A3B03882B193CC
:101A4200466BCF7A5448DD59622DEB3C700EF91F7C
:101A52008FF706E69DD414C5ABB122A0B9923083AC
:101A6200C77B4E6AD5585C49E33D6A2CF11E780F5C
:101A72000000C1C081C1400101C3C003800241C254
:101A820001C6C006800741C70005C1C581C4400424
:101A920001CCC00C800D41CD000FC1CF81CE400ED4
:101AA200000AC1CA81CB400B01C9C009800841C8E4
:101AB20001D8C018801941D9001BC1DB81DA401A54
:101AC200001EC1DE81DF401F01DDC01D801C41DC24
:101AD2000014C1D481D5401501D7C017801641D654
:101AE20001D2C012801341D30011C1D181D0401064
:101AF20001F0C030803141F10033C1F381F2403254
:101B02000036C1F681F7403701F5C035803441F423
:101B1200003CC1FC81FD403D01FFC03F803E41FED3
:101B220001FAC03A803B41FB0039C1F981F84038E3
:101B32000028C1E881E9402901EBC02B802A41EA53
:101B420001EEC02E802F41EF002DC1ED81EC402C23
:101B520001E4C024802541E50027C1E781E6402653
:101B62000022C1E281E3402301E1C021802041E063
:101B720001A0C060806141A10063C1A381A2406253
:101B82000066C1A681A7406701A5C065806441A423
:101B9200006CC1AC81AD406D01AFC06F806E41AED3
:101BA20001AAC06A806B41AB0069C1A981A84068E3
:101BB2000078C1B881B9407901BBC07B807A41BA53
:101BC20001BEC07E807F41BF007DC1BD81BC407C23
:101BD20001B4C074807541B50077C1B781B6407653
:101BE2000072C1B281B3407301B1C071807041B063
:101BF2000050C190819140510193C0538052419253
:101C02000196C056805741970055C1958194405422
:101C1200019CC05C805D419D005FC19F819E405ED2
:101C2200005AC19A819B405B0199C05980584198E2
:101C32000188C04880494189004BC18B818A404A52
:101C4200004EC18E818F404F018DC04D804C418C22
:101C52000044C184818540450187C0478046418652
:101C62000182C042804341830041C1818180404062
:101C7200EF92FF921F93CF93DF9300D000D0CDB7A6
:101C8200DEB79E012F5F3F4F41E06AE370E281E0E1
:101C92000E94A61311E089819A81892B09F410E030
:101CA200E12EF12CE982FA8282E090E00E94861E07
:101CB20090E0E816F90671F0612F82E090E00E9450
:101CC200A91D9E012F5F3F4F41E06AE370E281E070
:101CD2000E9453149E012F5F3F4F41E060E070E28B
:101CE20081E00E94A61384E090E00E94BC1E6981FC
:101CF2007A818617970721F084E090E00E94C11E46
:101D02009E012F5F3F4F41E061E070E281E00E945F
:101D1200A61386E090E00E94BC1E69817A81861734
:101D2200970721F086E090E00E94C11E9E012F5F7E
:101D32003F4F41E062E070E281E00E94A61388E03A
:101D420090E00E94BC1E69817A818617970721F074
:101D520088E090E00E94C11E9E012F5F3F4F41E04C
:101D620063E070E281E00E94A6138AE090E00E94A4
:101D7200BC1E69817A818617970721F08AE090E07C
:101D82000E94C11E9E012F5F3F4F41E069E370E256
:101D920081E00E94A61311E089819A81892B09F4BE
:101DA20010E0E12EF12CE982FA8283E090E00E94B9
:101DB200861E90E0E816F90609F1612F83E090E0B3
:101DC2000E94A91D9E012F5F3F4F41E069E370E22F
:101DD20081E00E94531489819A81892B49F58CE014
:101DE20090E00E94BC1E8B839C839E012D5F3F4F1F
:101DF20041E064E370E281E00E94531489819A8198
:101E0200892BB1F49E012F5F3F4F41E064E370E202
:101E120081E00E94A6138CE090E00E94BC1E6981C2
:101E22007A818617970721F08CE090E00E94C11E0C
:101E32002496CDBFDEBFDF91CF911F91FF90EF902F
:021E4200089501
:101E44008F929F92AF92BF92CF92DF92FF920F93A5
:101E54001F93CF93DF93B82E8B01F42EE9011882E0
:101E640019821A821B82642FC8010E942B1D8F3F86
:101E740009F4A6C0BB2009F44BC0FF2009F4A0C09C
:101E8400AF2DB0E01197A295B295B07FBA27A07F8D
:101E9400BA2720E030E0E82FF0E0EE0FFF1FEE0F4E
:101EA400FF1FEE0FFF1FBF016050784C6B01CB0189
:101EB4000496F60140815181B801641B750BAB0196
:101EC400420F531F440F551FFC0160817181460F5F
:101ED400571FFA014081518160E070E00A2E04C06E
:101EE400440F551F661F771F0A94D2F78880998084
:101EF400AA80BB80482959296A297B2948835983A8
:101F04006A837B832F5F3F4F50972F1590F258C001
:101F1400A82FB0E0FD01EE0FFF1FEE0FFF1FEE0F25
:101F2400FF1FE050F84C86819781892B09F448C043
:101F3400FF2009F445C0EF2DF0E03197E295F295CA
:101F4400F07FFE27E07FFE2720E030E0AA0FBB1FD2
:101F5400AA0FBB1FAA0FBB1FBD016050784C6B01B9
:101F6400CB010696D6014D915C91B801641B750BAB
:101F7400AB01420F531F440F551FDC016D917C913F
:101F8400460F571FDA014D915C9160E070E00E2E10
:101F940004C0440F551F661F771F0A94D2F7888028
:101FA4009980AA80BB80482959296A297B294883BA
:101FB40059836A837B832F5F3F4F70972F1590F26D
:101FC400DF91CF911F910F91FF90DF90CF90BF9041
:081FD400AF909F908F900895DB
:101FDC008F929F92AF92BF92CF92DF92EF92FF922D
:101FEC000F931F93CF93DF93F82E6B01142FE901FE
:101FFC00642FC6010E942B1D8F3F09F4A0C0FF2047
:10200C0009F448C0112309F49AC0A12EB12C21E087
:10201C00A21AB108AA0CBB1CAA0CBB1CAA0CBB1C98
:10202C00AA0CBB1CA0E0B0E0E82EF12CC701880F75
:10203C00991F880F991F880F991FFC01E050F84CCD
:10204C007F014F01F4E08F0E911CF701808191818B
:10205C00F601E81BF90BEA0FFB1F9F01220F331F40
:10206C00F40180819181F901E80FF91F28813981F0
:10207C004A815B816C817D818E819F810A2D0E94BA
:10208C00BB1C208331831196F0E1AF1AB108A11764
:10209C00E0F255C0A82EB12CF501EE0FFF1FEE0F8C
:1020AC00FF1FEE0FFF1FE050F84C86819781892BA4
:1020BC0009F445C0112309F442C0E12EF12C21E0B2
:1020CC00E21AF108EE0CFF1CEE0CFF1CEE0CFF1CD0
:1020DC00EE0CFF1CA0E0B0E0C501880F991F880F23
:1020EC00991F880F991FFC01E050F84C5F014F01BC
:1020FC00F6E08F0E911CF50180819181F601E81BB1
:10210C00F90BEA0FFB1F9F01220F331FF401808193
:10211C009181F901E80FF91F288139814A815B818E
:10212C006C817D818E819F810E2D0E94BB1C208332
:10213C0031831196F0E1EF1AF108A117E0F2DF916B
:10214C00CF911F910F91FF90EF90DF90CF90BF90A8
:08215C00AF909F908F90089551
:10216400EF92FF920F931F93CF93DF93CDB7DEB718
:102174002697CDBFDEBF9E012F5F3F4F41E06BE34B
:1021840070E281E00E94A61389819A81892B09F467
:10219400A1C086E0809305040E94521E0E941A1E6C
:1021A400E981FA818E01095F1F4FAE014D5F5F4FD8
:1021B40078019F01ADECBCEC0E94EF1D96958795CC
:1021C40096958795969587959C01220F331F880FC6
:1021D400991F880F991F880F991F820F931F9F01C2
:1021E400281B390BD7012E937D019F01ADECBCEC6C
:1021F4000E94EF1DFC01F695E795F695E795F69597
:10220400E7954E155F05A9F6E983FA83E0E4F4E067
:1022140084E08683BAEA21E134E0B15020403040C2
:10222400E1F7000085836AEA71E194E0615070404F
:102234009040E1F700008683AAEAB1E124E0A150CE
:10224400B0402040E1F70000858334E563E278E0A4
:10225400315060407040E1F700C000C094E022C0FB
:1022640080E09683AAEAB1E134E0A150B040304066
:10227400E1F7000095836AEA71E1A4E061507040DF
:10228400A040E1F700008F5F8213EBCFB9EA2BE7A0
:102294003CE1B15020403040E1F700C000C040179D
:1022A400510731F0DA012D91AD012111D9CFEECFD3
:1022B4000E94491E0E94BD1D86E080930604198277
:1022C4001A829E012F5F3F4F41E06BE370E281E091
:1022D4000E9453142696CDBFDEBFDF91CF911F918C
:0822E4000F91FF90EF900895A7
:1022EC00CF93DF9300D0CDB7DEB780E090E00E94B3
:1022FC00861E877F29F068E080E090E00E94A91D8F
:10230C0081E090E00E94861E982F9F7D39F08033EB
:10231C0029F060E081E090E00E94A91D88E090E047
:10232C000E94BC1E89839A83019631F461E272E0AB
:10233C0088E090E00E94C11E8AE090E00E94BC1EE2
:10234C0089839A83019631F460E372E08AE090E02D
:10235C000E94C11E82E090E00E94861E21E030E0C7
:10236C00811102C020E030E029833A839E012F5F67
:10237C003F4F41E06AE370E281E00E94531483E036
:10238C0090E00E94861E21E030E0811102C020E026
:10239C0030E029833A839E012F5F3F4F41E069E390
:1023AC0070E281E00E94531484E090E00E94BC1E15
:1023BC0089839A839E012F5F3F4F41E060E070E27A
:1023CC0081E00E94531486E090E00E94BC1E898339
:1023DC009A839E012F5F3F4F41E061E070E281E004
:1023EC000E94531488E090E00E94BC1E89839A835B
:1023FC009E012F5F3F4F41E062E070E281E00E945E
:10240C0053148AE090E00E94BC1E89839A839E013B
:10241C002F5F3F4F41E063E070E281E00E94531474
:10242C008CE090E00E94BC1E89839A839E012F5FF2
:10243C003F4F41E064E370E281E00E9453148EE070
:10244C0080930004E0E4F1E081ED808381E08283FD
:10245C009FEF93838783108611860F900F90DF91E7
:04246C00CF9108956F
:10247000CF92DF92EF92FF92CF93E0E0F4E080E31F
:10248000828381858063818789E0848B858B8185C8
:102490008063818780858073482F50E060E070E022
:1024A00009F04DC08091623A811149C081E080936A
:1024B000623A8091633A82958F709091633A2FEFE0
:1024C000280F223008F089C0C92FCF70C33008F020
:1024D00084C0813031F460E080E090E00E94A91D6A
:1024E00005C068E080E090E00E94A91DC11106C00F
:1024F00060E081E090E00E94A91D0DC0C13031F480
:1025000060E281E090E00E94A91D05C060E381E0E7
:1025100090E00E94A91D0E94E01B86E080930604C3
:10252000E0E0F4E096E097832AEA31E144E02150CC
:1025300030404040E1F700008150A9F74EC01092B2
:10254000623A403251056105710571F04031510523
:102550006105710589F00F2EF0E8CF2EF5E2DF2E30
:10256000E12CF12CF02D0FC00F2EC12CFBE4DF2E3F
:10257000E12CF12CF02D07C00F2EC12CF6E9DF2E37
:10258000E12CF12CF02DC701B6010E94331A9B01FA
:10259000AC0162E372ED83EC9CE40E94C61E20E075
:1025A00030E040E05FE30E94CA1E20E030E040E8F7
:1025B0005FE30E948F1E0E94851B6093280A709320
:1025C000290A68EA72EC82EA90E0A70196010E946B
:1025D000561C2093080830930908CF91FF90EF9084
:0625E000DF90CF9008958A
:1025E6008F929F92AF92BF92CF92DF92FF920F93FC
:1025F6001F93CF93DF93B82EEB01F42E8901642F3E
:10260600CE010E942B1D8F3F09F491C0BB2009F417
:1026160041C0FF2009F48BC04F2D50E041505109B5
:1026260042955295507F5427407F542720E030E052
:10263600A82FB0E0AA0FBB1FAA0FBB1FAA0FBB1F74
:10264600CD018050984C6C010496D6016D917C9119
:10265600FE01E61BF70BE20FF31FEE0FFF1FDC0177
:102666006D917C91E60FF71FD8018D909D90AD90EE
:10267600BC90042E04C0B694A794979487940A94A9
:10268600D2F7808291822F5F3F4F405151092F151B
:10269600E0F24DC0A82FB0E0FD01EE0FFF1FEE0FD8
:1026A600FF1FEE0FFF1FE050F84C86819781892BA4
:1026B600F1F1FF20E1F14F2D50E0415051094295D3
:1026C6005295507F5427407F542720E030E0AA0FD0
:1026D600BB1FAA0FBB1FAA0FBB1FFD01E050F84C82
:1026E6006F01CF010696D6016D917C91FE01E61B26
:1026F600F70BE20FF31FEE0FFF1FDC016D917C91CC
:10270600E60FF71FD8018D909D90AD90BC90042EDA
:1027160004C0B694A794979487940A94D2F78082BB
:1027260091822F5F3F4F405151092F15E0F2DF9103
:10273600CF911F910F91FF90DF90CF90BF90AF90F8
:062746009F908F900895A2
:10274C00CF92DF92EF92FF920F931F93CF93DF9371
:10275C00E82E8B01F42EE90118821982642FC8012E
:10276C000E942B1D8F3F09F48FC0EE2009F440C04E
:10277C00FF2009F489C04F2D50E04150510942957A
:10278C005295507F5427407F542720E030E0A82FEB
:10279C00B0E0AA0FBB1FAA0FBB1FAA0FBB1FCD0116
:1027AC008050984C6C010496D6016D917C91F80187
:1027BC00E61BF70BE20FF31FEE0FFF1FDC016D9111
:1027CC007C91E60FF71F60817181042E02C0660FA9
:1027DC00771F0A94E2F7E881F9816E2B7F2B6883CF
:1027EC0079832F5F3F4F405151092F15E8F24CC0B0
:1027FC00A82FB0E0FD01EE0FFF1FEE0FFF1FEE0F35
:10280C00FF1FE050F84C86819781892BE9F1FF205E
:10281C00D9F14F2D50E04150510942955295507FBE
:10282C005427407F542720E030E0AA0FBB1FAA0F8B
:10283C00BB1FAA0FBB1FFD01E050F84C6F01CF016D
:10284C000696D6016D917C91F801E61BF70BE20F11
:10285C00F31FEE0FFF1FDC016D917C91E60FF71F4C
:10286C0060817181042E02C0660F771F0A94E2F713
:10287C00E881F9816E2B7F2B688379832F5F3F4F23
:10288C00405151092F15E8F2DF91CF911F910F9113
:0A289C00FF90EF90DF90CF900895B9
:1028A600CF92DF92EF92FF920F931F93CF93DF9316
:1028B600E82EEB01F42E8901642FCE010E942B1D18
:1028C6008F3F09F488C0EE20E9F1FF2009F483C0A8
:1028D6004F2D50E04150510942955295507F542753
:1028E600407F542720E030E0A82FB0E0AA0FBB1F9E
:1028F600AA0FBB1FAA0FBB1FCD018050984C6C01BD
:102906000496D6016D917C91FE01E61BF70BE20F52
:10291600F31FEE0FFF1FDC016D917C91E60FF71F91
:10292600D8016D917C91042E02C0769567950A9424
:10293600E2F7608371832F5F3F4F405151092F1596
:1029460000F349C0A82FB0E0FD01EE0FFF1FEE0F08
:10295600FF1FEE0FFF1FE050F84C86819781892BF1
:10296600D1F1FF20C1F14F2D50E041505109429560
:102976005295507F5427407F542720E030E0AA0F1D
:10298600BB1FAA0FBB1FAA0FBB1FFD01E050F84CCF
:102996006F01CF010696D6016D917C91FE01E61B73
:1029A600F70BE20FF31FEE0FFF1FDC016D917C9119
:1029B600E60FF71FD8016D917C91042E02C0769523
:1029C60067950A94E2F7608371832F5F3F4F40510A
:1029D60051092F1500F3DF91CF911F910F91FF90B1
:0829E600EF90DF90CF900895FF
:1029EE0010C00E949C1E58F00E94951E40F029F4C3
:1029FE005F3F29F00C94B01E51110C94A41E0C9440
:102A0E00D71E0E94341C68F39923B1F3552391F31A
:102A1E00951B550BBB27AA2762177307840738F03F
:102A2E009F5F5F4F220F331F441FAA1FA9F335D09C
:102A3E000E2E3AF0E0E832D091505040E695001C50
:102A4E00CAF72BD0FE2F29D0660F771F881FBB1F0A
:102A5E00261737074807AB07B0E809F0BB0B802DE8
:102A6E00BF01FF2793585F4F3AF09E3F510578F014
:102A7E000C94B01E0C94A41E5F3FE4F3983ED4F366
:102A8E00869577956795B795F7959F5FC9F7880FE8
:102A9E00911D9695879597F90895E1E0660F771F3A
:102AAE00881FBB1F621773078407BA0720F0621BCB
:0E2ABE00730B840BBA0BEE1F88F7E09508959A
:102ACC000FC00E94951E38F00E949C1E20F095238A
:102ADC0011F00C94B01E0C94D71E11240C94A41E4F
:102AEC000E94341C70F3959FC1F3950F50E0551F55
:102AFC00629FF001729FBB27F00DB11D639FAA2747
:102B0C00F00DB11DAA1F649F6627B00DA11D661F95
:102B1C00829F2227B00DA11D621F739FB00DA11DB6
:102B2C00621F839FA00D611D221F749F3327A00D70
:102B3C00611D231F849F600D211D822F762F6A2F0C
:102B4C0011249F5750409AF0F1F088234AF0EE0F71
:102B5C00FF1FBB1F661F771F881F91505040A9F79E
:102B6C009E3F510580F00C94B01E0C94A41E5F3F48
:102B7C00E4F3983ED4F3869577956795B795F795DA
:102B8C00E7959F5FC1F7FE2B880F911D9695879552
:042B9C0097F9089508
:102BA000CF93DF93C0E0D4E080EC8A83E0E2F4E0EE
:102BB0008AE38283A0E4B4E089E012968C931297B2
:102BC00088E88E8B99E89F8B818B838B848B858B98
:102BD00050968C93509753969C9353978985806811
:102BE000898719968C911997886019968C931997F3
:102BF0003885488580852085C085F0851896DC91CC
:102C000018971896EC91441F4427441F8270842B18
:102C10003074432F50E055954795559547955595F8
:102C20004795482B2870822F90E095958795842BA7
:102C30009C2F9071990F982B8F2F8072880F880F7F
:102C4000892B6D2F617070E000247695679507944D
:102C5000769567950794762F602D682B8E2F887058
:0E2C6000880F682B6093633ADF91CF9108953F
:102C6E0011C00E94951E38F00E949C1E20F039F46F
:102C7E009F3F19F426F40C94D71E0EF4E095E7FB53
:102C8E000C94B01EE92F0E94341C58F3BA17620739
:102C9E0073078407950720F079F4A6F50C94A31E0C
:102CAE000EF4E0950B2EBA2FA02D0B01B901900159
:102CBE000C01CA01A0011124FF27591B99F0593F9D
:102CCE0050F4503E68F11A16F040A22F232F342FE5
:102CDE004427585FF3CF469537952795A795F04033
:102CEE005395C9F77EF41F16BA0B620B730B840B48
:102CFE00BAF09150A1F0FF0FBB1F661F771F881F00
:102D0E00C2F70EC0BA0F621F731F841F48F4879557
:102D1E0077956795B795F7959E3F08F0B0CF939549
:0E2D2E00880F08F09927EE0F97958795089566
:102D3C001F920F920FB60F9211240F931F932F9384
:102D4C003F934F935F936F937F938F939F93AF9327
:102D5C00BF93EF93FF93CF93DF9300D0CDB7DEB744
:102D6C0000E411E0F80183818160838381E0838337
:102D7C009E012F5F3F4F41E065E370E20E94A61376
:102D8C0089819A81019689839A839E012F5F3F4F97
:102D9C0041E065E370E281E00E945314F801838105
:102DAC008260838382E0838382818D7F82830E9411
:102DBC0038120E94D0150E94491E0E94BD1D86E04B
:102DCC00809306040F900F90DF91CF91FF91EF91BC
:102DDC00BF91AF919F918F917F916F915F914F9127
:102DEC003F912F911F910F910F900FBE0F901F903D
:022DFC00189528
:102DFE0000070E001A00026003000710001C0002FC
:102E0E00500000071F003C00026003000720003E38
:102E1E000002600304075100420001600000073306
:102E2E000064000260030007340066000260030FB6
:102E3E000751006A00016000010751006B0001603C
:102E4E0000000747008C00026003000748008E0058
:102E5E000260031A0751009400016000020751003E
:102E6E0095000160000008010000020460010008E6
:102E7E00020004020460010108010008020460015E
:102E8E00010802000C020460010208010010020495
:102E9E00600102080200140204600100016000419A
:0D2EAE002005000009000000412005000083
:102EBB000000AE005C010B02B90267031504C204EB
:102ECB006F051C06C80674071F08C90873091C0A7E
:102EDB00C40A6B0B120CB70C5C0DFF0DA20E430F4B
:102EEB00E30F82101F11BB115612F01287131E1421
:102EFB00B3144615D7156716F51682170C189518C7
:102F0B001B19A019231AA31A221B9F1B191C911CF6
:102F1B00071D7B1DEC1D5B1EC81E321F9A1FFF1F5A
:102F2B006220C22020217B21D4212A227D22CE2285
:102F3B001B236723AF23F52337247724B424EF24F3
:102F4B0026255B258C25BB25E6250F263526582601
:102F5B0078269426AE26C526D926E926F7260227FB
:062F6B0009270E271027C4
:102F7200AB01813011F4465A5F4F9A01A3E8BDE2DA
:102F82000E94EF1D0024880F991F001C880F991FB3
:102F9200001C892F902D68E671E0869F9001879F23
:102FA200300D969F300D1124CA01821B930B8B3575
:102FB200910540F4880F991FFC01E554F145808189
:102FC20091810895853B910558F4E4EBF0E0E81B0C
:102FD200F90BEE0FFF1FE554F145808191810895B1
:102FE2008F3021E0920758F4880F991FFC01ED5AA7
:102FF200F245808191819195819591090895E8E644
:10300200F1E0E81BF90BEE0FFF1FE554F14580815B
:0A301200918191958195910908952F
:10301C000F931F93CF93DF93082F192FD62F82E096
:10302C0080930504C0910608C07811F00E94521ECE
:10303C00E0E0FAE010A211A283E0808381E08093AB
:10304C00643A8091643A8111FCCFE0E0F8E086812B
:10305C00806486838481806484839FEF9D0FDD234D
:10306C0049F0A02FB12F848185FFFDCF8D918283F4
:10307C009150C8F7E0E0F8E0848186FFFDCFE0E0F6
:10308C00F8E086818F7B8683C1110E94491EE0E0A7
:10309C00FAE010A211A283E0808381E08093643A6D
:1030AC008091643A8111FCCF82E080930604DF9119
:0830BC00CF911F910F910895BF
:1030C400CF93DF9300D0CDB7DEB7E0E0F6E084E045
:1030D400828382E3848788E2808781E0808381E140
:1030E4008287868180FDFDCFE0E0F6E080818E7FDF
:1030F4008083A0E0B1E191962C91919790964C91A8
:1031040080899189A289B389B695A7959795879562
:10311400B695A79597958795022E000C330BBC01A5
:10312400621B730B9B01A42FB0E00E94EF1DDC0116
:10313400CB0180589F4FAF4FBF4F892F9A2FAB2F92
:10314400BB2789839A839E012F5F3F4F41E066E44A
:1031540070E281E00E9453140F900F90DF91CF91A1
:023164000895CC
:1031660088249924F401E401B0E49F93AA279A15D0
:103176008B049C04ED05FE05CF05D007A10798F446
:10318600AD2FDC2FCF2FFE2FE92D982C892E982FCF
:10319600872F762F652F542F432F322F2227B85093
:1031A60031F7BF9127C01B2EBF91BB27220F331FBC
:1031B600441F551F661F771F881F991F881C991C5F
:1031C600EE1FFF1FCC1FDD1FAA1FBB1F8A149B0407
:1031D600EC05FD05CE05DF05A007B10748F08A1806
:1031E6009B08EC09FD09CE09DF09A00BB10B216094
:1031F6001A94E1F62EF49401AF01BE01CD01000C44
:02320600089529
:10320800DF93CF931F930F939A9DF02D219FF00D7D
:103218008B9DF00D8A9DE02DF10D039FF00D029F0F
:10322800E00DF11D4E9DE00DF11D5E9DF00D4F9DD1
:10323800F00D7F936F93BF92AF925F934F93D50139
:103248000E94EF1D8B01AC01D7010E94EF1DEB011D
:10325800E80FF91FD6010E945B1E2F913F91D601FE
:103268000E94EF1DC60FD71FE81FF91FAF91BF912E
:103278000E945B1E2F913F910E94EF1DC60FD71F22
:10328800E81FF91FD6010E94EF1DE60FF71F9801EE
:10329800BE01CF0111240F911F91CF91DF910895A5
:1032A800CF93DF93CDB7DEB70E9476110E94EA195B
:1032B8000E94E01B0E94491E0E94601D0E94BD1DC5
:1032C80086E0E0E0F4E096E097832AEA31E144E022
:1032D800215030404040E1F700008150A9F7789430
:1032E8000E94D41E882311F1CDB6DEB60E94621862
:1032F8000E94D11E182F8DB79EB7811B91098DBFD3
:103308009EBF2DB73EB72F5F3F4F7901612FC9018F
:103318000E94521B612FC7010E946109803121F46C
:103328000E94390E0E94B210CDBEDEBE0E94CE1E93
:0A3338008823B1F20E947400D3CF85
:103342000F931F93CF93DF938D30F0F5A82FB0E04A
:10335200FD01EE0FFF1FEE0FFF1FEE0FFF1FE050EC
:10336200F84C86819781009779F1FD01EE0FFF1FDE
:10337200EE0FFF1FEE0FFF1FE050F84C2481358146
:10338200268337838483958320E030E0DF01BF0109
:103392006A5F7F4F8F010E5F1F4FA901440F551FB8
:1033A200EB01E881F981E40FF51F108211822F5F92
:1033B2003F4FF801408151818D919C911197481B9B
:1033C200590B4217530748F7DF91CF911F910F9185
:0233D20008955C
:1033D400EF92FF920F931F93CF93DF93CDB7DEB796
:1033E4002A97CDBFDEBFE0E0F1E12485838590E03C
:1033F400922B89839A832285818590E0922B8B83FB
:103404009C832085878190E0922B8D839E832681E7
:10341400858190E0922B8F8398872481838190E02B
:10342400922B89879A87CE0101967C010CE310E2E6
:10343400970141E0B80181E00E9453140F5F1F4FD0
:1034440092E0E90EF11C013480E2180789F72A960C
:10345400CDBFDEBFDF91CF911F910F91FF90EF9011
:023464000895C9
:10346600E89409C097FB3EF4909580957095619518
:103476007F4F8F4F9F4F9923A9F0F92F96E9BB27CE
:103486009395F695879577956795B795F111F8CF4A
:10349600FAF4BB0F11F460FF1BC06F5F7F4F8F4FB5
:1034A6009F4F16C0882311F096E911C0772321F0AB
:1034B6009EE8872F762F05C0662371F096E8862F43
:1034C60070E060E02AF09A95660F771F881FDAF79A
:0A34D600880F9695879597F90895E1
:1034E0000F931F93CF93DF938D3078F5A82FB0E023
:1034F000FD01EE0FFF1FEE0FFF1FEE0FFF1FE0504D
:10350000F84C86819781892B01F120E030E0DF01C2
:10351000BF016A5F7F4F8F010E5F1F4FA901440FEC
:10352000551FEB01E881F981E40FF51F108211822C
:103530002F5F3F4FF801408151818D919C911197F0
:10354000481B590B4217530748F7DF91CF911F9142
:043550000F9108953A
:103554001F920F920FB60F9211242F933F934F9304
:103564005F936F937F938F939F93AF93BF93CF9307
:10357400DF93EF93FF93C0E0D4E08FEF89870E943D
:103584001A1E0E94521EE0E4F1E0808591850396A4
:103594008487958782818260828386E08D83FF9110
:1035A400EF91DF91CF91BF91AF919F918F917F91D7
:1035B4006F915F914F913F912F910F900FBE0F909C
:0435C4001F901895A7
:1035C8002091613A261710F46091613A662399F0C8
:1035D800AC012FEF260F30E02F5F3F4F280F391F28
:1035E800FC01DF01A41BB50BA458B64C8C91819348
:1035F800E217F307B1F78091613A861B8093613A2D
:103608008091613A882399F020E070E0822F90E061
:10361800FB01E80FF91FE458F64C3081FC01E4582F
:10362800F64C30832F5F8091613A281778F308951C
:103638001F920F920FB60F9211242F933F934F931F
:103648005F936F937F938F939F93AF93BF93EF9302
:10365800FF938FEF809349040E941A1E0E94521E06
:10366800E0E4F1E0808591850396848795878281DF
:103678008260828386E080930504FF91EF91BF9179
:10368800AF919F918F917F916F915F914F913F91F2
:0C3698002F910F900FBE0F901F901895FF
:1036A4002091663A261710F46091663A662361F019
:1036B400E82FF92F80E090E0DC01AC5BB54C2C9155
:1036C400219301968617C0F38091663A861B8093F6
:1036D400663A8091663A882399F020E070E0822F60
:1036E40090E0FB01E80FF91FEC5BF54C3081FC0125
:1036F400EC5BF54C30832F5F8091663A281778F3A2
:063704001092653A0895E1
:10370A000E943C1C88F09F5798F0B92F9927B7510F
:10371A00B0F0E1F0660F771F881F991F1AF0BA956B
:10372A00C9F714C0B13091F00E94A31EB1E0089508
:10373A000C94A31E672F782F8827B85F39F0B93FFA
:10374A00CCF3869577956795B395D9F73EF490951E
:0E375A008095709561957F4F8F4F9F4F08951A
:103768001F921FB61F9211248F93EF93FF9382E04D
:10377800809305048091663A803110F01092663A81
:10378800E091663A81E08E0F8093663AF0E080918E
:103798000008EC5BF54C8083E0E0FAE010A211A28F
:1037A80083E0808382E080930604FF91EF918F91FC
:0837B8001F901FBE1F90189521
:1037C0000F931F93CF93DF93E0E2F4E082E08283D4
:1037D00081E08183D8E0D28B0E9438120E94D015FC
:1037E00000E018E089E0F801858381E090E00E9424
:1037F000861EC82F80E090E00E94861E8C2B83607E
:10380000F8018783D68380E180930A0ADF91CF9104
:063810001F910F910895C5
:103816001F921FB61F9211248F93EF93FF9384E09C
:10382600809305048091613A803210F01092613ADB
:10383600E091613A81E08E0F8093613AF0E08091E9
:103846002008E458F64C8083E0E8FAE012861386F6
:1038560083E08083FF91EF918F911F901FBE1F9091
:023866001895B3
:1038680057FD9058440F551F59F05F3F71F0479529
:10387800880F97FB991F61F09F3F79F0879508950E
:10388800121613061406551FF2CF4695F1DF08C02D
:10389800161617061806991FF1CF8695710561054A
:0438A80008940895E3
:1038AC00A1E21A2EAA1BBB1BFD010DC0AA1FBB1F38
:1038BC00EE1FFF1FA217B307E407F50720F0A21BAA
:1038CC00B30BE40BF50B661F771F881F991F1A9417
:1038DC0069F760957095809590959B01AC01BD0141
:0438EC00CF0108956B
:1038F0001F921FB61F9211248F93EF93FF93E0E066
:10390000FAE08FEF838710821092643A8091663AD2
:10391000863028F41092663A1092653A03C081E02E
:103920008093653AFF91EF918F911F901FBE1F907A
:023930001895E8
:103932008091613A8823D9F080917C399091613AE3
:1039420091509093613A9091613A992381F090E07D
:10395200292F30E0F901E358F64C4081F901E4588F
:10396200F64C40839F5F2091613A921788F3089545
:1039720097FB10F8169400080F93083098F008503F
:10398200232F342F452F562F672F782F892F902DD5
:10399200F4CF0594979587957795679557954795B1
:0C39A200379527950A95AAF70F91089514
:1039AE002091613A261710F46091613A662399F0DE
:1039BE00AC016150262F30E02F5F3F4F280F391F8B
:1039CE00FC01DF01A41BB50BA458B64C8C9181935E
:0839DE00E217F307B1F70895A9
:1039E600409550952FEF260F662391F0A82FB92FFB
:1039F600ED91652F77274E27E42FF0E0EE0FFF1F9E
:103A0600EE58F7464081518146275727215080F7C7
:083A1600CA0180959095089506
:103A1E002FEF260F6623A9F0A82FB92F842F952FED
:103A2E00ED91492F55278E27E82FF0E0EE0FFF1F5F
:103A3E00EE58F5468081918184279527215080F795
:083A4E000895842F952F0895BF
:103A5600AC01E0E0F8E390E08FEF9A01260F311D0C
:103A6600B90161507109208131814217530730F045
:103A7600228133812617370708F0892F9F5F3896F2
:063A86009C3089F7089551
:103A8C001F921FB61F9211248F93EF93FF93E0E8C0
:103A9C00FAE08FEF868310821092613A1092603AAE
:103AAC0084E080930604FF91EF918F911F901FBECD
:043ABC001F901895AA
:103AC000E0E4F4E082E0828388E0818B84E0858317
:103AD0008183E0EEF5E0828184608283E0E2F8E0B9
:103AE00087E594E0808791871582168283E087833B
:023AF000089537
:103AF2000F93083090F0982F872F762F652F542F31
:103B0200432F322F22270850F4CF220F331F441F96
:103B1200551F661F771F881F991F0A95B2F70F91CD
:023B2200089504
:103B2400052E97FB1EF400940E94761E57FD07D0C5
:103B34000E94561C07FC03D04EF40C94761E50953C
:0E3B44004095309521953F4F4F4F5F4F0895AC
:103B5200262FAF93BF93E0E0F0E1328131FDFDCF3C
:103B6200DC01A050BC4E2C932DE924BF23E020831E
:083B72000196BF91AF91089587
:103B7A00E0E2F8E0858180688583868180688683B3
:103B8A00E0E8FAE08FEF86831286138682E0858367
:023B9A0008958C
:103B9C00092E0394000C11F4882352F0BB0F40F44F
:103BAC00BF2B11F460FF04C06F5F7F4F8F4F9F4F8F
:023BBC0008956A
:103BBE00609570958095909530954095509521958E
:103BCE003F4F4F4F5F4F6F4F7F4F8F4F9F4F089518
:103BDE00A29FB001B39FC001A39F700D811D112440
:0E3BEE00911DB29F700D811D1124911D08952F
:103BFC009091613A981720F49091603A9111F8CF16
:0C3C0C009091603A81E0911180E00895F1
:103C1800689401C0E8948F929F92CF93DF930E949B
:0C3C2800B318DF91CF919F908F9008950A
:103C3400E0E2F8E085818F77858386818F778683BC
:0A3C44001092603A1092850A08956C
:103C4E000024A7FD00942A17300540055005600595
:083C5E00700580059005089532
:103C66000E94EF1DA59F900DB49F900DA49F800DFF
:063C7600911D11240895C8
:103C7C00EC010E94DF1E0E94DE1ECE010E94E01E9F
:063C8C00CE010E94DC1EC7
:103C9200E0E0F8E08581806885838681806886839C
:023CA200089583
:103CA400E0E0F8E085818F77858386818F7786834E
:023CB400089571
:103CB6000E94EF1D460F571FC81FD91F08F43196E3
:023CC60008955F
:103CC8002A0D3B1D4C1D5D1D6E1D7F1D801F911F04
:023CD80008954D
:103CDA002A193B094C095D096E097F09800B910B72
:023CEA0008953B
:103CEC0090958095709561957F4F8F4F9F4F08955C
:103CFC00B7FF0C94331E0E94331E821B930B089546
:103D0C0003D0808199270895FC01E050FC4E089562
:0E3D1C005058BB27AA270E9437160C94CE1DC4
:0E3D2A0000240A9416161706180609060895B6
:0E3D380000240A9412161306140605060895B8
:0E3D4600E894BB2766277727CB0197F90895ED
:0C3D54008091613A811180917C390895C2
:0C3D600097F99F6780E870E060E008952C
:0C3D6C00EE0FFF1F0590F491E02D09946C
:0A3D78000E948A1E80819181089547
:0A3D82000E94A91D272F0C94AA1D12
:083D8C000E94F7140C94CE1DF7
:083D94000E9466150C94CE1D7F
:063D9C008091613A0895D8
:063DA2008091663A0895CD
:063DA8008091653A0895C8
:063DAE009FEF80EC089578
:043DB4000C9400006B
:043DB8000E947200F3
:023DBC00089568
:023DBE00089566
:023DC000089564
:103DC20000000700FC390C3A10001300343A3C3A68
:103DD20018001D001C3A283A28002F00DC39EC3963
:103DE2003800420028393E3950005700BC39CC39DE
:103DF20060006B00F838103978007F009C39AC39CC
:103E020088009500C038DC3800021702603890380C
:103E120000200320543A0000342047205439000087
:02000004008278
:0900000000007D0000F6FF000085
:02000004008377
:01000000C53A
:00000001FF
